:10000000F128FF3FFF3FFF3FFF00030E8301BD00CC
:100010000408BC000A08BE008A017008C1008501FE
:100020008701860120088316850083122108831624
:1000300087008312220886002F08233F84000008CF
:10004000A200301C2628F030A20528280F30A20577
:1000500005302F0203185228FF30A1002F08003A64
:10006000031D35283D30A00086282F08013A031DC6
:100070003C283B30A00086282F08023A031D432865
:100080003730A00086282F08033A031D4A282F3056
:10009000A00086282F08043A031D51281F30A00015
:1000A000862886283F30A0002F08053A031D5B28CC
:1000B000FE30A10086282F08063A031D6228FD3075
:1000C000A10086282F08073A031D6928FB30A100EC
:1000D00086282F08083A031D7028F730A1008628CB
:1000E0002F08093A031D7728EF30A10086282F0832
:1000F0000A3A031D7E28DF30A10086282F080B3A1C
:10010000031D86283E30A000FF30A100AF0A0C304E
:100110002F02031C8D28AF01B00A0B114108F0001B
:100120003E088A003C0884003D0E8300FF0E7F0ECF
:100130000900031383124008003A031DA228BB30B4
:10014000C000E3284008013A031DA9288230C000FE
:10015000E3284008023A031DB0283E30C000E328DF
:100160004008033A031DB728AE30C000E32840081A
:10017000043A031DBE288730C000E3284008053A32
:10018000031DC528AD30C000E3284008063A031D12
:10019000CC289D30C000E3284008073A031DD3282F
:1001A000A230C000E3284008083A031DDA28BF3017
:1001B000C000E3284008093A031DE128A730C00029
:1001C000E3282030C0003F080B3C0318E9280B301F
:1001D000BF003F08233FF000700884004008800003
:1001E0000800031383129F01073083169F008312B8
:1001F00085013F30831685008312860183168601B0
:1002000083128701FF30831687008B0189308100BC
:1002100001308312900007309200AF010130B1002D
:100220000230B200B301B401B501B601B701B801A3
:100230000130B9000830A3000130BF003108C00010
:1002400099200230BF003208C00099200430A60077
:100250000430BF003308C00099200530BF003408C7
:10026000C00099200430A9000730BF003508C00045
:1002700099200830BF003608C00099200430AC0037
:100280000A30BF003708C00099200B30BF00380883
:10029000C0009920A0308B00071B8B29B20A0A30BE
:1002A0003202031C5529B201B10A3108013A031D7B
:1002B00064293208023A031D64293908031D6329A1
:1002C0000130B9006429B9013108013A031D6F29D1
:1002D0003208033A031D6F29B1010130B200390819
:1002E000031975290830A30077292030A3000130B5
:1002F000BF003108C00099200230BF003208C000A2
:100300009920071F81298F01C8300F0203188B29FC
:10031000071F81298429871BC529B40A0A303402A2
:10032000031C9929B401B30A06303302031C99292E
:10033000B301B501B601B701B8010430BF003308FD
:10034000C00099200530BF003408C0009920073054
:10035000BF003508C00099200830BF003608C00033
:1003600099200A30BF003708C00099200B30BF0029
:100370003808C0009920871FBB298F01C8300F02A1
:100380000318C529871FBB29BE298C1C5D2A8C1028
:1003900000303A07F1003B080318013F043FF20028
:1003A0007108BA007208BB0027307202031DDA29F7
:1003B00010307102031C5D2A1030BA02031CBB030B
:1003C0002730BB02B80A0A303802031CFB29B801E7
:1003D000B70A0A303702031CFB29B701B60A0A30F4
:1003E0003602031CFB29B601B50A06303502031C90
:1003F000FB29B501B40A0A303402031C272AB401D0
:10040000B30A06303302031C272AB301B20A0A30AA
:100410003202031C0D2AB201B10A3108013A031D50
:100420001C2A3208023A031D1C2A3908031D1B2A04
:100430000130B9001C2AB9013108013A031D272AED
:100440003208033A031D272AB1010130B2003908EE
:1004500003192D2A0830A3002F2A2030A3000130D1
:10046000BF003108C00099200230BF003208C00030
:1004700099200430A6000430BF003308C000992042
:100480000530BF003408C00099200430A9000730AF
:10049000BF003508C00099200830BF003608C000F2
:1004A00099200430AC000A30BF003708C000992002
:1004B0000B30BF003808C00099204C295E2AFF3F4E
:02400E00723FFF
:00000001FF
